:100000000C9466000C9483000C9483000C94830081
:100010000C9483000C9483000C9483000C94830054
:100020000C9483000C9483000C9483000C94830044
:100030000C9483000C94F5040C9483000C948300BE
:100040000C9483000C9483000C9483000C94830024
:100050000C9483000C9483000C9483000C94830014
:100060000C9483000C9483000C9483000C94830004
:100070000C9483000C9483000C9483000C948300F4
:100080000C9483000C9483000C9483000C948300E4
:100090000C9483000C9483000C9483000C948300D4
:1000A0000C9483000C9483000C9483000C948300C4
:1000B0000C9483000C9483000C9483000C948300B4
:1000C0000C9483000C9483000C94830011241FBEB5
:1000D000CFEFD8E0DEBFCDBF11E0A0E0B1E0ECE1B2
:1000E000F5E102C005900D92A83DB107D9F721E0D6
:1000F000A8EDB1E001C01D92AA3DB207E1F70E9450
:10010000A1020C948C0A0C940000CF93DF93CDB71E
:10011000DEB780E890E0FC01108281E890E028E002
:10012000FC01208384E890E0FC0111821082000031
:10013000DF91CF910895CF93DF93CDB7DEB784E8F9
:1001400090E0FC011182108288E890E029E03DE314
:10015000FC013183208386E390E0FC018081882FBD
:1001600090E082709927892B49F086E390E026E39E
:1001700030E0F90120812260FC01208381E890E0D9
:1001800021E830E0F90120812560FC012083000096
:10019000DF91CF910895CF93DF93CDB7DEB786E39C
:1001A00090E0FC018081882F90E082709927892B54
:1001B00049F086E390E026E330E0F90120812260F7
:1001C000FC0120838FE690E028E0FC012083000002
:1001D000DF91CF910895CF93DF93CDB7DEB786E35C
:1001E00090E0FC018081882F90E08270992721E0C7
:1001F000892B09F420E0822FDF91CF910895CF93CE
:10020000DF9300D0CDB7DEB787E690E09A8389838D
:1002100088EC90E0FC01108289EC90E028E1FC0180
:1002200020838AEC90E026E0FC01208389819A817A
:100230008DEC90E0FC0110828CEC90E029813A81F9
:10024000FC01208300000F900F90DF91CF91089563
:10025000CF93DF931F92CDB7DEB789838EEC90E00A
:100260002981FC012083000088EC90E0FC01808162
:10027000882F90E080749927892BB1F388EC90E067
:1002800028EC30E0F90120812064FC01208300008B
:100290000F90DF91CF910895CF93DF93CDB7DEB765
:1002A000000088EC90E0FC0180818823D4F78EEC7C
:1002B00090E0FC018081DF91CF910895CF93DF938F
:1002C00000D000D0CDB7DEB79C838B831A82198211
:1002D0000FC089819A812B813C81820F931FFC0181
:1002E00080810E94280189819A8101969A8389835D
:1002F00089819A812B813C81820F931FFC0180812F
:10030000882339F700000F900F900F900F90DF9126
:10031000CF910895CF93DF93CDB7DEB78CE290E015
:10032000FC018081882F90E080749927892B11F43B
:1003300084E006C080E290E0FC0180818095837FAC
:10034000DF91CF910895CF93DF93CDB7DEB7639759
:100350000FB6F894DEBF0FBECDBF898B7B8B6A8B47
:100360001A8219828989882F90E084709927892BB5
:1003700011F080E289838989837F8A838BE290E010
:100380002BE230E0F90130812A812327FC01208310
:100390008EE290E02EE230E0F901308129812327BE
:1003A000FC01208320E030E040E85EE364EA70ED89
:1003B00084EA93E40E9425064A895B8928EE33E0AB
:1003C000429FC001439F900D529F900D1124CC017C
:1003D000A0E0B0E0BC01CD010E944008DC01CB01EF
:1003E0008B839C83AD83BE8320E030E04AE755E4F5
:1003F0006B817C818D819E810E943809DC01CB015B
:100400008F839887A987BA8720E030E040E85FE3D0
:100410006F81788589859A850E94930788232CF4BB
:1004200081E090E09C878B873FC020E03FEF4FE763
:1004300057E46F81788589859A850E94330918165B
:100440004CF520E030E040E251E46B817C818D810D
:100450009E810E943809DC01CB01BC01CD010E94C4
:100460001108DC01CB019C878B870FC080E991E0EC
:100470009E878D878D859E850197F1F79E878D8755
:100480008B859C8501979C878B878B859C85892B89
:1004900069F714C06F81788589859A850E94110853
:1004A000DC01CB019C878B878B859C85988B8F8704
:1004B0008F8598890197F1F7988B8F878BE290E071
:1004C0002BE230E0F90130812A812327FC012083CF
:1004D0008EE290E02EE230E0F9013081298123277D
:1004E000FC012083000063960FB6F894DEBF0FBEB8
:1004F000CDBFDF91CF910895CF93DF93CDB7DEB716
:1005000081E290E0FC01108282E290E02FEFFC019A
:1005100020838AE290E02FEFFC0120838BE290E0C1
:100520002FEFFC0120838DE290E020E3FC0120838B
:100530008EE290E02FEFFC0120830000DF91CF914D
:1005400008958F929F92AF92BF92CF92DF92EF92D7
:10055000FF92CF93DF93CDB7DEB7E3970FB6F89452
:10056000DEBF0FBECDBFF8940E9485000E947C02C2
:100570000E94FF001A82198280E191E00E945E01D0
:1005800007C00E944C01882F90E0C0979A8389830E
:1005900089819A810497ACF789819A811816190686
:1005A00084F716C289819A8182309105D9F083300F
:1005B000910569F1019709F03FC083E090E09E83C7
:1005C0008D8383E090E09C838B8385E090E0988727
:1005D0008F8383E090E09A87898785E090E09C870D
:1005E0008B872AC084E090E09E838D8382E090E038
:1005F0009C838B8387E090E098878F8383E090E0F3
:100600009A8789878AE090E09C878B8715C085E070
:1006100090E09E838D8381E090E09C838B838AE0D1
:1006200090E098878F8385E090E09A8789878FE0B4
:1006300090E09C878B8700001E861D86188A1F8687
:100640001A8A198A7FC189859A85092E000CAA0BFE
:10065000BB0BBC01CD010E9442086B017C012B85C4
:100660003C8589859A85A901481B590BCA01092E29
:10067000000CAA0BBB0BBC01CD010E9442084B0130
:100680005C018D819E810197092E000CAA0BBB0B8A
:10069000BC01CD010E944208DC01CB019C01AD01EF
:1006A000C501B4010E949807DC01CB014C015D013A
:1006B00089899A89092E000CAA0BBB0BBC01CD01BC
:1006C0000E944208DC01CB019C01AD01C501B401CF
:1006D0000E943809DC01CB01BC01CD010E947C07DE
:1006E000DC01CB019C01AD01C701B6010E941007DE
:1006F000DC01CB01BC01CD010E940A08DC01CB0169
:100700009B8F8A8F1C8A1B8A37C00E94190A27E098
:1007100030E0B9010E94A5098D8B8D89833011F4D9
:1007200087E08D8B8D89282F30E081E090E002C03A
:10073000880F991F2A95E2F78C8F8AE00E94280182
:100740008D89805D0E9428018AE00E9428019E0117
:10075000215D3F4F8B899C89820F931F2C8DFC015B
:1007600020838B819C81BC018C8D0E94A3018B898D
:100770009C8901969C8B8B8B2B893C898A8D9B8DC8
:100780002817390714F28F8198859093D9018093A7
:10079000D8010E949B00198E188EC7C086E691E092
:1007A0000E945E010E94EB008823C1F08091D80175
:1007B0009091D90101979093D9018093D8010E941B
:1007C000CB000E949B002DEC3CEC4CEC5DE364EA1A
:1007D00070ED82E893E40E94250606C00E948A011B
:1007E000882F90E09F8B8E8B8E899F89892B39F47F
:1007F0008091D8019091D901181619069CF280E0D9
:1008000090E0AAE7B3E489A39AA3ABA3BCA320E03A
:1008100030E04AE755E469A17AA18BA19CA10E942E
:100820003809DC01CB018DA39EA3AFA3B8A720E0BC
:1008300030E040E85FE36DA17EA18FA198A50E9402
:10084000930788232CF481E090E09AA789A73FC002
:1008500020E03FEF4FE757E46DA17EA18FA198A55F
:100860000E94330918164CF520E030E040E251E4D4
:1008700069A17AA18BA19CA10E943809DC01CB015E
:10088000BC01CD010E941108DC01CB019AA789A708
:100890000FC080E991E09CA78BA78BA59CA5019731
:1008A000F1F79CA78BA789A59AA501979AA789A775
:1008B00089A59AA5892B69F714C06DA17EA18FA186
:1008C00098A50E941108DC01CB019AA789A789A5E8
:1008D0009AA59EA78DA78DA59EA50197F1F79EA726
:1008E0008DA78D859E8501969E878D879E01215DB2
:1008F0003F4F888D998D820F931FFC018081282F97
:1009000030E08E899F892817390741F48F859889AF
:100910000196988B8F870E94310502C00E9447057F
:10092000888D998D0196998F888F288D398D8A8D24
:100930009B8D281739070CF431CF89899A89019644
:100940009A8B898B29893A898D819E81281739074D
:100950000CF479CE8F859889092E000CAA0BBB0B5D
:10096000BC01CD010E9442086B017C018D859E85F2
:10097000092E000CAA0BBB0BBC01CD010E94420842
:10098000DC01CB019C01AD01C701B6010E949807B3
:10099000DC01CB018D8F9E8FAF8FB8A32DEC3CEC8B
:1009A0004CE45FE36D8D7E8D8F8D98A10E9433099D
:1009B000882354F089819A8101969A83898380E8FB
:1009C00091E00E945E0104C00E940506000005C07F
:1009D00089819A8103970CF4E5CD89819A810397E7
:1009E0000CF4C8CD0E94E505C5CD1F920F92009072
:1009F0005F000F9211242F933F934F935F936F9358
:100A00007F938F939F93AF93BF93EF93FF93CF9376
:100A1000DF93CDB7DEB78091D8019091D9019C01C9
:100A2000215031093093D9012093D80118161906A5
:100A30001CF00E942506FDCF0000DF91CF91FF91B1
:100A4000EF91BF91AF919F918F917F916F915F9146
:100A50004F913F912F910F9000925F000F901F9048
:100A60001895CF93DF93CDB7DEB78DE891E00E9464
:100A70005E012DEC3CEC4CEC5DE360E070E08CED55
:100A800093E40E9425060000DF91CF910895CF9353
:100A9000DF93CDB7DEB72E970FB6F894DEBF0FBE4B
:100AA000CDBF88E991E00E945E012DEC3CEC4CE466
:100AB0005EE36CE57FEC82E893E40E94250680E02B
:100AC00090E0A8ECB1E489839A83AB83BC8320E0F7
:100AD00030E04AE755E469817A818B819C810E94EC
:100AE0003809DC01CB018D839E83AF83B88720E07A
:100AF00030E040E85FE36D817E818F8198850E94C0
:100B0000930788232CF481E090E09A8789873FC07F
:100B100020E03FEF4FE757E46D817E818F8198851C
:100B20000E94330918164CF520E030E040E251E411
:100B300069817A818B819C810E943809DC01CB011B
:100B4000BC01CD010E941108DC01CB019A87898785
:100B50000FC080E991E09C878B878B859C850197EE
:100B6000F1F79C878B8789859A8501979A87898772
:100B700089859A85892B69F714C06D817E818F8163
:100B800098850E941108DC01CB019A8789878985A5
:100B90009A859E878D878D859E850197F1F79E8723
:100BA0008D872DEC3CEC4CE45EE36CE57FEC82E859
:100BB00093E40E94250600002E960FB6F894DEBF3F
:100BC0000FBECDBFDF91CF910895CF93DF93CDB707
:100BD000DEB78BEA91E00E945E0120E030E040E069
:100BE0005FE360E070E083E893E40E94250620E084
:100BF00030E040E05FE360E070E084EC93E40E946A
:100C000025060000DF91CF910895CF93DF93CDB7F4
:100C1000DEB780EC91E00E945E0120E030E040E031
:100C20005FE360E070E085EA93E40E94250620E03F
:100C300030E040E05FE360E070E083E993E40E942D
:100C400025060000DF91CF910895CF93DF93CDB7B4
:100C5000DEB76E970FB6F894DEBF0FBECDBF6F8BB9
:100C6000788F898F9A8F2B8F3C8F4D8F5E8F2F8936
:100C7000388D498D5A8D60E070E080E89FE30E94D6
:100C80009807DC01CB0120E030E040E050E4BC01FB
:100C9000CD010E949807DC01CB0120E030E04AE75B
:100CA00054E4BC01CD010E943809DC01CB018B83E7
:100CB0009C83AD83BE832F89388D498D5A8D60E02A
:100CC00070E080E89FE30E949807DC01CB019C0163
:100CD000AD016B8D7C8D8D8D9E8D0E949807DC0102
:100CE000CB01BC01CD010E940A08DC01CB01988731
:100CF0008F831A82198281C08B819C81AD81BE81D4
:100D000089879A87AB87BC8720E030E04AE755E4C3
:100D100069857A858B859C850E943809DC01CB0129
:100D20008D879E87AF87B88B20E030E040E85FE397
:100D30006D857E858F8598890E94930788232CF482
:100D400081E090E09A8B898B3FC020E03FEF4FE736
:100D500057E46D857E858F8598890E943309181622
:100D60004CF520E030E040E251E469857A858B85DE
:100D70009C850E943809DC01CB01BC01CD010E9499
:100D80001108DC01CB019A8B898B0FC080E991E0BF
:100D90009C8B8B8B8B899C890197F1F79C8B8B8B20
:100DA00089899A8901979A8B898B89899A89892B54
:100DB00069F714C06D857E858F8598890E9411081A
:100DC000DC01CB019A8B898B89899A899E8B8D8BCB
:100DD0008D899E890197F1F79E8B8D8B8EE290E035
:100DE0002EE230E0F901308120E12327FC0120834D
:100DF00089819A8101969A8389838F819885298137
:100E00003A812817390708F477CF00006E960FB69D
:100E1000F894DEBF0FBECDBFDF91CF91089550583B
:100E2000BB27AA270E9427070C94E1080E94D30839
:100E300038F00E94DA0820F039F49F3F19F426F4C4
:100E40000C94D0080EF4E095E7FB0C94A108E92F70
:100E50000E94F20858F3BA176207730784079507D0
:100E600020F079F4A6F50C942C090EF4E0950B2EE5
:100E7000BA2FA02D0B01B90190010C01CA01A001EC
:100E80001124FF27591B99F0593F50F4503E68F147
:100E90001A16F040A22F232F342F4427585FF3CF88
:100EA000469537952795A795F0405395C9F77EF459
:100EB0001F16BA0B620B730B840BBAF09150A1F0A2
:100EC000FF0FBB1F661F771F881FC2F70EC0BA0F28
:100ED000621F731F841F48F4879577956795B795B0
:100EE000F7959E3F08F0B0CF9395880F08F09927AB
:100EF000EE0F9795879508950E94140990F09F37FB
:100F000048F4911116F40C942D0960E070E080E82B
:100F10009FE3089526F01B16611D711D811D0C9421
:100F2000A7080C94C2080E947D0808F481E0089587
:100F30000E94AC070C94E1080E94DA0858F00E9465
:100F4000D30840F029F45F3F29F00C94A108511117
:100F50000C942D090C94D0080E94F20868F3992390
:100F6000B1F3552391F3951B550BBB27AA276217A5
:100F70007307840738F09F5F5F4F220F331F441FB2
:100F8000AA1FA9F335D00E2E3AF0E0E832D09150E6
:100F90005040E695001CCAF72BD0FE2F29D0660FD3
:100FA000771F881FBB1F261737074807AB07B0E816
:100FB00009F0BB0B802DBF01FF2793585F4F3AF01C
:100FC0009E3F510578F00C94A1080C942D095F3FC9
:100FD000E4F3983ED4F3869577956795B795F795A2
:100FE0009F5FC9F7880F911D9695879597F908958A
:100FF000E1E0660F771F881FBB1F62177307840726
:10100000BA0720F0621B730B840BBA0BEE1F88F734
:10101000E09508950E9411086894B1110C942D096F
:1010200008950E94FA0888F09F5798F0B92F9927E1
:10103000B751B0F0E1F0660F771F881F991F1AF0C3
:10104000BA95C9F714C0B13091F00E942C09B1E0F3
:1010500008950C942C09672F782F8827B85F39F0F2
:10106000B93FCCF3869577956795B395D9F73EF45C
:1010700090958095709561957F4F8F4F9F4F089504
:10108000E89409C097FB3EF4909580957095619522
:101090007F4F8F4F9F4F9923A9F0F92F96E9BB27D8
:1010A0009395F695879577956795B795F111F8CF54
:1010B000FAF4BB0F11F460FF1BC06F5F7F4F8F4FBF
:1010C0009F4F16C0882311F096E911C0772321F0B5
:1010D0009EE8872F762F05C0662371F096E8862F4D
:1010E00070E060E02AF09A95660F771F881FDAF7A4
:1010F000880F9695879597F90895990F0008550FD1
:10110000AA0BE0E8FEEF16161706E807F907C0F08D
:1011100012161306E407F50798F0621B730B840B95
:10112000950B39F40A2661F0232B242B252B21F46F
:1011300008950A2609F4A140A6958FEF811D811D0F
:10114000089597F99F6780E870E060E0089588232C
:1011500071F4772321F09850872B762F07C06623F0
:1011600011F499270DC09051862B70E060E02AF0B1
:101170009A95660F771F881FDAF7880F96958795DF
:1011800097F908959F3F31F0915020F48795779516
:101190006795B795880F911D9695879597F908954E
:1011A0009FEF80EC089500240A941616170618067F
:1011B0000906089500240A9412161306140605065B
:1011C0000895092E0394000C11F4882352F0BB0FEC
:1011D00040F4BF2B11F460FF04C06F5F7F4F8F4F4F
:1011E0009F4F089557FD9058440F551F59F05F3F8A
:1011F00071F04795880F97FB991F61F09F3F79F039
:1012000087950895121613061406551FF2CF4695BA
:10121000F1DF08C0161617061806991FF1CF86953C
:1012200071056105089408950E94FA08A0F0BEE7D0
:10123000B91788F4BB279F3860F41616B11D672FC5
:10124000782F8827985FF7CF869577956795B11D9A
:1012500093959639C8F30895E894BB2766277727B6
:10126000CB0197F908950E947D0808F48FEF089547
:101270000E944B090C94E1080E94D30838F00E94A8
:10128000DA0820F0952311F00C94A1080C94D008F2
:1012900011240C942D090E94F20870F3959FC1F35C
:1012A000950F50E0551F629FF001729FBB27F00D14
:1012B000B11D639FAA27F00DB11DAA1F649F662769
:1012C000B00DA11D661F829F2227B00DA11D621FB8
:1012D000739FB00DA11D621F839FA00D611D221F72
:1012E000749F3327A00D611D231F849F600D211D56
:1012F000822F762F6A2F11249F5750409AF0F1F0D9
:1013000088234AF0EE0FFF1FBB1F661F771F881F41
:1013100091505040A9F79E3F510580F00C94A108D0
:101320000C942D095F3FE4F3983ED4F386957795AE
:101330006795B795F795E7959F5FC1F7FE2B880FE7
:10134000911D9695879597F9089597FB072E16F4AA
:10135000009407D077FD09D00E94B90907FC05D099
:101360003EF4909581959F4F0895709561957F4FBC
:101370000895AA1BBB1B51E107C0AA1FBB1FA617DC
:10138000B70710F0A61BB70B881F991F5A95A9F72E
:1013900080959095BC01CD0108958F929F92AF9258
:1013A000BF92CF92DF92EF92FF92CF93DF93EC0147
:1013B000688179818A819B8161157105810591051B
:1013C00021F464E279ED8BE597E02DE133EF41E024
:1013D00050E00E94290A49015A019B01AC01A7EA89
:1013E000B1E40E94480A6B017C01ACEEB4EFA501A8
:1013F00094010E94560ADC01CB018C0D9D1DAE1D8F
:10140000BF1DB7FF03C00197A109B0488883998326
:10141000AA83BB839F77DF91CF91FF90EF90DF90FE
:10142000CF90BF90AF909F908F9008950E94CD096C
:10143000089580E091E00E94CD090895A0E0B0E019
:101440008093000190930101A0930201B0930301E6
:101450000895052E97FB1EF400940E94400A57FD44
:1014600007D00E945B0A07FC03D04EF40C94400A9C
:1014700050954095309521953F4F4F4F5F4F0895C0
:1014800090958095709561957F4F8F4F9F4F0895F0
:101490000E947D0AA59F900DB49F900DA49F800D82
:1014A000911D11240895B7FF0C94480A0E94480A20
:1014B000821B930B0895A1E21A2EAA1BBB1BFD01F0
:1014C0000DC0AA1FBB1FEE1FFF1FA217B307E40723
:1014D000F50720F0A21BB30BE40BF50B661F771F7B
:1014E000881F991F1A9469F760957095809590955B
:1014F0009B01AC01BD01CF010895A29FB001B39F34
:10150000C001A39F700D811D1124911DB29F700D0C
:0C151000811D1124911D0895F894FFCF57
:10151C000100000074696D657220746573740A00B3
:10152C0053494D4F4E2047414D450A456E746572E7
:10153C0020796F7572207374617274696E672064A0
:10154C006966666963756C7479206C6576656C3A4E
:10155C000A312E20456173790A322E204D6F646555
:10156C00726174650A332E2047697665206D65209B
:10157C007061696E2E000A676F7420656C656D650D
:10158C006E742C2077616974696E672E2E2E0A009A
:10159C000A6E657874206C6576656C0A000A436F78
:1015AC007272656374210A000A496E636F72726508
:1015BC0063742067756573732E0A000A596F752062
:1015CC0062656174207468652067616D65210A002D
:1015DC000A596F75206C6F6F73652C2074727920AB
:0815EC00616761696E3F0A00AE
:00000001FF
